:020000040000FA
:06000000FBEF00F012000E
:06002A0001000E020000BF
:08003000800000001000000038
:08003800816A806A070EC16EA7
:100040001F0E926E936A80A808D08050816E010EB8
:10005000E66EE4EC00F0E55266D0816A4B0EE66E87
:10006000E4EC00F0E55200019A6B080EE76E9A1975
:10007000E8AE02D0E73402D0E7509A5D14E280B8CF
:1000800012D0010E9AC0E7FFE75204E0E846FE0BEB
:10009000E706FCE1816E4B0EE66EE4EC00F0E55203
:1000A00000019A2BE2D79A6B080EE76E9A19E8AE18
:1000B00002D0E73402D0E7509A5D15E280B813D041
:1000C0009A29046E010E045204E0E846FE0B040671
:1000D000FCE1FF0F816E4B0EE66EE4EC00F0E552A2
:1000E00000019A2BE1D79A6B100EE76E9A19E8AED1
:1000F00002D0E73402D0E7509A5D15E280B813D001
:100100009AC0E9FFEA6AE9BEEA68800EE926000EB5
:10011000EA22EF50816E4B0EE66EE4EC00F0E55201
:0A01200000019A2BE1D78FD71200DF
:06012A002A0EF66E000E25
:10013000F76E000EF86E00010900F550956F09008A
:10014000F550966F03E1956701D03DD00900F55059
:10015000906F0900F550916F0900F550926F0900FA
:100160000900F550E96E0900F550EA6E0900090032
:100170000900F550936F0900F550946F09000900CC
:10018000F6CF97F0F7CF98F0F8CF99F090C0F6FF40
:1001900091C0F7FF92C0F8FF0001935302E194531E
:1001A00007E00900F550EE6E9307F8E29407F9D7DF
:1001B00097C0F6FF98C0F7FF99C0F8FF00019507B8
:0801C000000E965BBFD7120090
:0801C800FF0EE350036EEF0E81
:1001D00001D0F30EE76EE72EEBEF00F00C0E026E8F
:1001E000E76AE72EF1EF00F0022EF0EF00F0032EA9
:0601F000E9EF00F012002F
:0A01F60015EE00F025EE00F0F86AA7
:0E020000019C95EC00F01CEC00F0FDD7120004
:02020E003F06A9
:0E0210005B4F666D7D077F6F777C395E79717D
:020000040030CA
:0E00000000220F0E000181000FC00FE00F4024
:00000001FF
